 can

 Timestamp is 4da2a530 (Mon Apr 11 18:52:32 2011)

 Preferred load address is 10000000

 Start         Length     Name                   Class
 0001:00000000 00000004H .CRT$XCA                CODE
 0001:00000004 00000004H .CRT$XCZ                CODE
 0001:00000008 00000004H .CRT$XIA                CODE
 0001:0000000c 00000004H .CRT$XIZ                CODE
 0001:00000010 00000004H .CRT$XPA                CODE
 0001:00000014 00000004H .CRT$XPZ                CODE
 0001:00000018 00000004H .CRT$XTA                CODE
 0001:0000001c 00000004H .CRT$XTZ                CODE
 0001:00000020 00001b1cH .rdata                  CODE
 0001:00001b3c 00000020H .rdata$debug            CODE
 0001:00001b5c 00004bccH .text                   CODE
 0001:00006728 00000048H .xdata                  CODE
 0001:00006770 0000003cH .idata$2                CODE
 0001:000067ac 00000014H .idata$3                CODE
 0001:000067c0 000000c0H .idata$4                CODE
 0001:00006880 000000a6H .idata$6                CODE
 0001:00006930 00000102H .edata                  CODE
 0002:00000000 000000c0H .idata$5                DATA
 0002:000000c0 0000044cH .data                   DATA
 0002:0000050c 00000010H .bss                    DATA
 0003:00000000 00000220H .pdata                  DATA

  Address         Publics by Value              Rva+Base       Lib:Object

 0000:00000000       ___safe_se_handler_table   00000000     <absolute>
 0000:00000000       ___safe_se_handler_count   00000000     <absolute>
 0001:00000000       __xc_a                     10001000     corelib0:crt0init.obj
 0001:00000004       __xc_z                     10001004     corelib0:crt0init.obj
 0001:00000008       __xi_a                     10001008     corelib0:crt0init.obj
 0001:0000000c       __xi_z                     1000100c     corelib0:crt0init.obj
 0001:00000010       __xp_a                     10001010     corelib0:crt0init.obj
 0001:00000014       __xp_z                     10001014     corelib0:crt0init.obj
 0001:00000018       __xt_a                     10001018     corelib0:crt0init.obj
 0001:0000001c       __xt_z                     1000101c     corelib0:crt0init.obj
 0001:00000040       ??_C@_1FO@JLECKMND@?$AAB?$AAS?$AAP?$AAC?$AAA?$AAN?$AAC?$AAl?$AAo?$AAc?$AAk?$AAC?$AAo?$AAn?$AAf?$AAi?$AAg?$AA?3?$AA?5?$AAD?$AAi?$AAs?$AAa?$AAb?$AAl?$AAe?$AA?5?$AAC?$AAA?$AAN?$AA?5?$AAc@ 10001040     bspcan.obj
 0001:000000a0       ??_C@_1FM@MLHKOMKJ@?$AAB?$AAS?$AAP?$AAC?$AAA?$AAN?$AAC?$AAl?$AAo?$AAc?$AAk?$AAC?$AAo?$AAn?$AAf?$AAi?$AAg?$AA?3?$AA?5?$AAE?$AAn?$AAa?$AAb?$AAl?$AAe?$AA?5?$AAC?$AAA?$AAN?$AA?5?$AAc?$AAl@ 100010a0     bspcan.obj
 0001:00000100       ??_C@_1GG@HHDDEKFK@?$AAB?$AAS?$AAP?$AAS?$AAe?$AAt?$AAC?$AAa?$AAn?$AAP?$AAo?$AAw?$AAe?$AAr?$AAE?$AAn?$AAa?$AAb?$AAl?$AAe?$AA?3?$AA?5?$AAD?$AAD?$AAK?$AAG?$AAp?$AAi?$AAo?$AAW?$AAr?$AAi@ 10001100     bspcan.obj
 0001:00000168       ??_C@_1CI@OHCJFJPM@?$AAE?$AAR?$AAR?$AAO?$AAR?$AA?3?$AA?5?$AA?$CF?$AAs?$AA?5?$AAl?$AAi?$AAn?$AAe?$AA?5?$AA?$CF?$AAd?$AA?3?$AA?5?$AA?$AA@ 10001168     bspcan.obj
 0001:00000190       ??_C@_1JI@GEFPGOFA@?$AAc?$AA?3?$AA?2?$AAw?$AAi?$AAn?$AAc?$AAe?$AAr?$AAo?$AAo?$AAt?$AAs?$AA?2?$AAt?$AAo?$AAp?$AAa?$AAz?$AA?2?$AAw?$AAi?$AAn?$AAc?$AAe?$AA7?$AA0?$AA0?$AA?2?$AAp?$AAl?$AAa@ 10001190     bspcan.obj
 0001:00000228       ??_C@_1CO@JOOMHEJL@?$AAC?$AAA?$AAN?$AA_?$AAI?$AAn?$AAi?$AAt?$AA?5?$AA?9?$AA?5?$AAh?$AAD?$AAe?$AAv?$AA?$DN?$AA0?$AAx?$AA?$CF?$AAx?$AA?$AN?$AA?6?$AA?$AA@ 10001228     can_common_topaz_v1:can_io.obj
 0001:00000258       ??_C@_1EO@EKPNPFED@?$AAC?$AAA?$AAN?$AA_?$AAI?$AAn?$AAi?$AAt?$AA?3?$AA?5?$AA?5?$AAR?$AAe?$AAg?$AAQ?$AAu?$AAe?$AAr?$AAy?$AAV?$AAa?$AAl?$AAu?$AAe?$AAE?$AAx?$AA?5?$AAf?$AAa?$AAi?$AAl?$AAe@ 10001258     can_common_topaz_v1:can_io.obj
 0001:000002a8       ??_C@_1M@EENNDIOJ@?$AAI?$AAn?$AAd?$AAe?$AAx?$AA?$AA@ 100012a8     can_common_topaz_v1:can_io.obj
 0001:000002b8       ??_C@_1EK@EINOINMC@?$AAC?$AAA?$AAN?$AA_?$AAI?$AAn?$AAi?$AAt?$AA?3?$AA?5?$AA?5?$AAO?$AAp?$AAe?$AAn?$AAD?$AAe?$AAv?$AAi?$AAc?$AAe?$AAK?$AAe?$AAy?$AA?5?$AAf?$AAa?$AAi?$AAl?$AAe?$AAd?$AA?$CB@ 100012b8     can_common_topaz_v1:can_io.obj
 0001:00000304       ??_C@_1BK@PNCCHPI@?$AAC?$AAA?$AAN?$AA_?$AAI?$AAn?$AAi?$AAt?$AA?5?$AA?$CL?$AA?$AN?$AA?6?$AA?$AA@ 10001304     can_common_topaz_v1:can_io.obj
 0001:00000320       ??_C@_1BO@LEHOMHHC@?$AAC?$AAA?$AAN?$AA_?$AAD?$AAe?$AAi?$AAn?$AAi?$AAt?$AA?5?$AA?9?$AA?$AN?$AA?6?$AA?$AA@ 10001320     can_common_topaz_v1:can_io.obj
 0001:00000340       ??_C@_1EC@FHFBAALP@?$AAC?$AAA?$AAN?$AA_?$AAD?$AAe?$AAi?$AAn?$AAi?$AAt?$AA?5?$AA?$CL?$AAD?$AAe?$AAv?$AAi?$AAc?$AAe?$AAC?$AAo?$AAn?$AAt?$AAe?$AAx?$AAt?$AA?$DN?$AA0?$AAx?$AA?$CF?$AAx?$AA?$AN?$AA?6@ 10001340     can_common_topaz_v1:can_io.obj
 0001:00000384       ??_C@_1BK@MNLOMOHP@?$AAC?$AAA?$AAN?$AA_?$AAO?$AAp?$AAe?$AAn?$AA?5?$AA?9?$AA?$AN?$AA?6?$AA?$AA@ 10001384     can_common_topaz_v1:can_io.obj
 0001:000003a0       ??_C@_1EA@MMEMBCAA@?$AAC?$AAA?$AAN?$AA_?$AAO?$AAp?$AAe?$AAn?$AA?5?$AA?$CL?$AAh?$AAD?$AAe?$AAv?$AAi?$AAc?$AAe?$AAC?$AAo?$AAn?$AAt?$AAe?$AAx?$AAt?$AA?$DN?$AA0?$AAx?$AA?$CF?$AAx?$AA?$AN?$AA?6?$AA?$AA@ 100013a0     can_common_topaz_v1:can_io.obj
 0001:000003e0       ??_C@_1BM@MGBMFAAI@?$AAC?$AAA?$AAN?$AA_?$AAC?$AAl?$AAo?$AAs?$AAe?$AA?5?$AA?9?$AA?$AN?$AA?6?$AA?$AA@ 100013e0     can_common_topaz_v1:can_io.obj
 0001:000003fc       ??_C@_1BM@HDFJIP@?$AAC?$AAA?$AAN?$AA_?$AAC?$AAl?$AAo?$AAs?$AAe?$AA?5?$AA?$CL?$AA?$AN?$AA?6?$AA?$AA@ 100013fc     can_common_topaz_v1:can_io.obj
 0001:00000418       ??_C@_1CE@CHGJALAB@?$AAC?$AAA?$AAN?$AA_?$AAI?$AAO?$AAC?$AAo?$AAn?$AAt?$AAr?$AAo?$AAl?$AA?5?$AA?9?$AA?$AN?$AA?6?$AA?$AA@ 10001418     can_common_topaz_v1:can_io.obj
 0001:00000440       ??_C@_1FI@DPGIPHAK@?$AAE?$AAx?$AAc?$AAe?$AAp?$AAt?$AAi?$AAo?$AAn?$AA?5?$AAi?$AAn?$AA?5?$AAC?$AAA?$AAN?$AA?5?$AAI?$AAO?$AAC?$AAT?$AAL?$AA_?$AAP?$AAO?$AAW?$AAE?$AAR?$AA_?$AAC?$AAA?$AAP@ 10001440     can_common_topaz_v1:can_io.obj
 0001:00000498       ??_C@_1FK@FLBIPJMP@?$AAE?$AAx?$AAc?$AAe?$AAp?$AAt?$AAi?$AAo?$AAn?$AA?5?$AAi?$AAn?$AA?5?$AAC?$AAS?$AAP?$AAI?$AA?5?$AAI?$AAO?$AAC?$AAT?$AAL?$AA_?$AAP?$AAO?$AAW?$AAE?$AAR?$AA_?$AAC?$AAA@ 10001498     can_common_topaz_v1:can_io.obj
 0001:000004f8       ??_C@_1LG@ICHCLBCJ@?$AAc?$AA?3?$AA?2?$AAw?$AAi?$AAn?$AAc?$AAe?$AAr?$AAo?$AAo?$AAt?$AAs?$AA?2?$AAt?$AAo?$AAp?$AAa?$AAz?$AA?2?$AAw?$AAi?$AAn?$AAc?$AAe?$AA7?$AA0?$AA0?$AA?2?$AAp?$AAl?$AAa@ 100014f8     can_common_topaz_v1:can_io.obj
 0001:000005b0       ??_C@_1DG@EMILGBPI@?$AAC?$AAA?$AAN?$AA_?$AAI?$AAO?$AAC?$AAT?$AAL?$AA_?$AAS?$AAE?$AAT?$AA_?$AAC?$AAA?$AAN?$AA_?$AAM?$AAO?$AAD?$AAE?$AA?5?$AA?9?$AA?$AN?$AA?6?$AA?$AA@ 100015b0     can_common_topaz_v1:can_io.obj
 0001:000005e8       ??_C@_1BO@MJFJLNLG@?$AAG?$AAe?$AAt?$AA?5?$AAM?$AAo?$AAd?$AAe?$AA?5?$AA?3?$AA?$CF?$AAx?$AA?$AN?$AA?6?$AA?$AA@ 100015e8     can_common_topaz_v1:can_io.obj
 0001:00000608       ??_C@_1DG@IKOEGIHP@?$AAC?$AAA?$AAN?$AA_?$AAI?$AAO?$AAC?$AAT?$AAL?$AA_?$AAS?$AAE?$AAT?$AA_?$AAC?$AAA?$AAN?$AA_?$AAM?$AAO?$AAD?$AAE?$AA?5?$AA?$CL?$AA?$AN?$AA?6?$AA?$AA@ 10001608     can_common_topaz_v1:can_io.obj
 0001:00000640       ??_C@_1DA@ECMLOCPH@?$AAC?$AAA?$AAN?$AA_?$AAI?$AAO?$AAC?$AAo?$AAn?$AAt?$AAr?$AAo?$AAl?$AA?3?$AAR?$AAE?$AAS?$AAE?$AAT?$AA?5?$AA?9?$AA?$AN?$AA?6?$AA?$AA@ 10001640     can_common_topaz_v1:can_io.obj
 0001:00000670       ??_C@_1DA@IEKEOLHA@?$AAC?$AAA?$AAN?$AA_?$AAI?$AAO?$AAC?$AAo?$AAn?$AAt?$AAr?$AAo?$AAl?$AA?3?$AAR?$AAE?$AAS?$AAE?$AAT?$AA?5?$AA?$CL?$AA?$AN?$AA?6?$AA?$AA@ 10001670     can_common_topaz_v1:can_io.obj
 0001:000006a0       ??_C@_1EK@CJKDNJNP@?$AAC?$AAA?$AAN?$AA_?$AAI?$AAO?$AAC?$AAo?$AAn?$AAt?$AAr?$AAo?$AAl?$AA?3?$AAC?$AAA?$AAN?$AA_?$AAI?$AAO?$AAC?$AAT?$AAL?$AA_?$AAT?$AAR?$AAA?$AAN?$AAS?$AAF?$AAE?$AAR@ 100016a0     can_common_topaz_v1:can_io.obj
 0001:000006f0       ??_C@_1HC@OGHDMNBN@?$AAC?$AAA?$AAN?$AA_?$AAI?$AAO?$AAC?$AAo?$AAn?$AAt?$AAr?$AAo?$AAl?$AA?3?$AAp?$AAM?$AAa?$AAr?$AAs?$AAh?$AAa?$AAl?$AAl?$AAe?$AAd?$AA_?$AAp?$AAt?$AAr?$AA?5?$AAp?$AAM@ 100016f0     can_common_topaz_v1:can_io.obj
 0001:00000768       ??_C@_1GI@MACIIFHC@?$AAC?$AAA?$AAN?$AA_?$AAI?$AAO?$AAC?$AAo?$AAn?$AAt?$AAr?$AAo?$AAl?$AA?3?$AAp?$AAM?$AAa?$AAr?$AAs?$AAh?$AAa?$AAl?$AAl?$AAe?$AAd?$AA_?$AAp?$AAt?$AAr?$AA?5?$AAp?$AAM@ 10001768     can_common_topaz_v1:can_io.obj
 0001:000007d0       ??_C@_1GA@ILDHOADA@?$AAC?$AAA?$AAN?$AA_?$AAI?$AAO?$AAC?$AAo?$AAn?$AAt?$AAr?$AAo?$AAl?$AA?3?$AAp?$AAM?$AAa?$AAr?$AAs?$AAh?$AAa?$AAl?$AAl?$AAe?$AAd?$AA_?$AAp?$AAt?$AAr?$AA?5?$AAC?$AAA@ 100017d0     can_common_topaz_v1:can_io.obj
 0001:00000830       ??_C@_1GC@KFMPPNMI@?$AAC?$AAA?$AAN?$AA_?$AAI?$AAO?$AAC?$AAo?$AAn?$AAt?$AAr?$AAo?$AAl?$AA?3?$AAp?$AAM?$AAa?$AAr?$AAs?$AAh?$AAa?$AAl?$AAl?$AAe?$AAd?$AA_?$AAp?$AAt?$AAr?$AA?5?$AAC?$AAA@ 10001830     can_common_topaz_v1:can_io.obj
 0001:00000898       ??_C@_1FA@NNMBLML@?$AAi?$AAN?$AAu?$AAm?$AAP?$AAa?$AAc?$AAk?$AAe?$AAt?$AAs?$AA?3?$AA?$CF?$AAd?$AA?5?$AA?5?$AA?5?$AAp?$AAP?$AAa?$AAc?$AAk?$AAe?$AAt?$AAs?$AA?$FL?$AA0?$AA?$FN?$AA?4?$AAb?$AAy?$AAR@ 10001898     can_common_topaz_v1:can_io.obj
 0001:000008e8       ??_C@_1EA@KJMCLANI@?$AAC?$AAA?$AAN?$AA_?$AAI?$AAO?$AAC?$AAo?$AAn?$AAt?$AAr?$AAo?$AAl?$AA?3?$AAG?$AAE?$AAT?$AA_?$AAC?$AAL?$AAO?$AAC?$AAK?$AA_?$AAR?$AAA?$AAT?$AAE?$AA?5?$AA?$AN?$AA?6?$AA?$AA@ 100018e8     can_common_topaz_v1:can_io.obj
 0001:00000928       ??_C@_1EC@MPCBOOFE@?$AAC?$AAA?$AAN?$AA_?$AAI?$AAO?$AAC?$AAo?$AAn?$AAt?$AAr?$AAo?$AAl?$AA?3?$AAG?$AAE?$AAT?$AA_?$AAC?$AAL?$AAO?$AAC?$AAK?$AA_?$AAR?$AAA?$AAT?$AAE?$AA?5?$AA?$CL?$AA?$AN?$AA?6@ 10001928     can_common_topaz_v1:can_io.obj
 0001:00000970       ??_C@_1EI@MDMMAPGN@?$AAC?$AAA?$AAN?$AA_?$AAI?$AAO?$AAC?$AAo?$AAn?$AAt?$AAr?$AAo?$AAl?$AA?3?$AA?5?$AA?$CL?$AAh?$AAO?$AAp?$AAe?$AAn?$AAC?$AAo?$AAn?$AAt?$AAe?$AAx?$AAt?$AA?$DN?$AA0?$AAx?$AA?$CF@ 10001970     can_common_topaz_v1:can_io.obj
 0001:000009b8       ??_C@_1GK@DHDAKADL@?$AAC?$AAA?$AAN?$AA_?$AAD?$AAl?$AAl?$AAE?$AAn?$AAt?$AAr?$AAy?$AA?3?$AA?5?$AAD?$AAL?$AAL?$AA_?$AAP?$AAR?$AAO?$AAC?$AAE?$AAS?$AAS?$AA_?$AAD?$AAE?$AAT?$AAA?$AAC?$AAH@ 100019b8     can_common_topaz_v1:can_io.obj
 0001:00000a28       ??_C@_1GK@HDLFIMMN@?$AAC?$AAA?$AAN?$AA_?$AAD?$AAl?$AAl?$AAE?$AAn?$AAt?$AAr?$AAy?$AA?3?$AA?5?$AAD?$AAL?$AAL?$AA_?$AAP?$AAR?$AAO?$AAC?$AAE?$AAS?$AAS?$AA_?$AAA?$AAT?$AAT?$AAA?$AAC?$AAH@ 10001a28     can_common_topaz_v1:can_io.obj
 0001:00000a94       ??_7?$Buffer_t@VDuplicateTraits_t@detail@marshal@ce@@@detail@marshal@ce@@6B@ 10001a94     can_common_topaz_v1:can_io.obj
 0001:00000a98       ??_C@_1FO@DDBELOJM@?$AA?$CF?$AAs?$AA?3?$AA?5?$AAc?$AAr?$AAe?$AAa?$AAt?$AAe?$AA?5?$AAC?$AAA?$AAN?$AA?5?$AAI?$AAS?$AAT?$AA?5?$AAt?$AAh?$AAr?$AAe?$AAa?$AAd?$AA?5?$AAs?$AAu?$AAc?$AAc?$AAe?$AAs@ 10001a98     can_common_topaz_v1:canclass.obj
 0001:00000af8       ??_C@_1EI@BPFOGHHH@?$AA?$CF?$AAs?$AA?3?$AA?5?$AAc?$AAr?$AAe?$AAa?$AAt?$AAe?$AA?5?$AAC?$AAA?$AAN?$AA?5?$AAI?$AAS?$AAT?$AA?5?$AAt?$AAh?$AAr?$AAe?$AAa?$AAd?$AA?5?$AAs?$AAu?$AAc?$AAc?$AAe?$AAs@ 10001af8     can_common_topaz_v1:canclass.obj
 0001:00000b40       ??_C@_1DG@IKMOEBDF@?$AA?$CF?$AAs?$AA?3?$AA?5?$AAC?$AAr?$AAe?$AAa?$AAt?$AAe?$AAT?$AAh?$AAr?$AAe?$AAa?$AAd?$AA?5?$AAf?$AAa?$AAi?$AAl?$AAe?$AAd?$AA?$CB?$AA?$AN?$AA?6?$AA?$AA@ 10001b40     can_common_topaz_v1:canclass.obj
 0001:00000b78       ??_C@_1CG@JKDBKNHM@?$AAC?$AAA?$AAN?$AAC?$AAl?$AAa?$AAs?$AAs?$AA?3?$AA?3?$AAC?$AAA?$AAN?$AAC?$AAl?$AAa?$AAs?$AAs?$AA?$AA@ 10001b78     can_common_topaz_v1:canclass.obj
 0001:00000ba0       ??_C@_1JA@NIBDIJHO@?$AAC?$AAA?$AAN?$AAC?$AAl?$AAa?$AAs?$AAs?$AA?3?$AA?3?$AAC?$AAA?$AAN?$AAC?$AAl?$AAa?$AAs?$AAs?$AA?3?$AAI?$AAn?$AAt?$AAe?$AAr?$AAr?$AAu?$AAp?$AAt?$AAi?$AAn?$AAi?$AAt@ 10001ba0     can_common_topaz_v1:canclass.obj
 0001:00000c30       ??_C@_1FM@LKLAJDNF@?$AAC?$AAA?$AAN?$AA_?$AAI?$AAn?$AAi?$AAt?$AA?3?$AAK?$AAe?$AAr?$AAn?$AAe?$AAl?$AAI?$AAo?$AAC?$AAo?$AAn?$AAt?$AAr?$AAo?$AAl?$AA?$CI?$AA?$CJ?$AA?3?$AA?5?$AAd?$AAw?$AAS?$AAy@ 10001c30     can_common_topaz_v1:canclass.obj
 0001:00000c90       ??_C@_1IA@DJFKHOHG@?$AAC?$AAA?$AAN?$AA_?$AAI?$AAn?$AAi?$AAt?$AA?3?$AAK?$AAe?$AAr?$AAn?$AAe?$AAl?$AAI?$AAo?$AAC?$AAo?$AAn?$AAt?$AAr?$AAo?$AAl?$AA?$CI?$AA?$CJ?$AA?3?$AAI?$AAO?$AAC?$AAT?$AAL@ 10001c90     can_common_topaz_v1:canclass.obj
 0001:00000d10       ??_C@_1IC@JMLPAFED@?$AAC?$AAA?$AAN?$AA_?$AAI?$AAn?$AAi?$AAt?$AA?3?$AAK?$AAe?$AAr?$AAn?$AAe?$AAl?$AAI?$AAo?$AAC?$AAo?$AAn?$AAt?$AAr?$AAo?$AAl?$AA?$CI?$AA?$CJ?$AA?3?$AA?5?$AAI?$AAR?$AAQ?$AA?5@ 10001d10     can_common_topaz_v1:canclass.obj
 0001:00000d98       ??_C@_1FE@FNBIAAGE@?$AAC?$AAA?$AAN?$AA_?$AAI?$AAn?$AAi?$AAt?$AA?3?$AAC?$AAr?$AAe?$AAa?$AAt?$AAe?$AAE?$AAv?$AAe?$AAn?$AAt?$AA?$CI?$AA?$CJ?$AA?3?$AA?5?$AAh?$AAR?$AAe?$AAv?$AAE?$AAv?$AAe?$AAn@ 10001d98     can_common_topaz_v1:canclass.obj
 0001:00000df0       ??_C@_1FK@NECCHALK@?$AAC?$AAA?$AAN?$AA_?$AAI?$AAn?$AAi?$AAt?$AA?3?$AAC?$AAr?$AAe?$AAa?$AAt?$AAe?$AAE?$AAv?$AAe?$AAn?$AAt?$AA?$CI?$AA?$CJ?$AA?3?$AA?5?$AAh?$AAI?$AAn?$AAt?$AAe?$AAr?$AAr?$AAu@ 10001df0     can_common_topaz_v1:canclass.obj
 0001:00000e50       ??_C@_1KI@PFIDLPDO@?$AAC?$AAA?$AAN?$AA_?$AAI?$AAn?$AAi?$AAt?$AA?3?$AAC?$AAr?$AAe?$AAa?$AAt?$AAe?$AAE?$AAv?$AAe?$AAn?$AAt?$AA?$CI?$AA?$CJ?$AA?3?$AA?5?$AAI?$AAn?$AAt?$AAe?$AAr?$AAr?$AAu?$AAp@ 10001e50     can_common_topaz_v1:canclass.obj
 0001:00000ef8       ??_C@_1FC@EEMDKIAI@?$AAC?$AAA?$AAN?$AA_?$AAI?$AAn?$AAi?$AAt?$AA?3?$AAM?$AAm?$AAM?$AAa?$AAp?$AAI?$AAo?$AAS?$AAp?$AAa?$AAc?$AAe?$AA?$CI?$AA?$CJ?$AA?3?$AA?5?$AAp?$AAC?$AAA?$AAN?$AAr?$AAe?$AAg@ 10001ef8     can_common_topaz_v1:canclass.obj
 0001:00000f50       ??_C@_1FO@MNIDIFLN@?$AAC?$AAA?$AAN?$AA_?$AAI?$AAn?$AAi?$AAt?$AA?3?$AAM?$AAm?$AAM?$AAa?$AAp?$AAI?$AAo?$AAS?$AAp?$AAa?$AAc?$AAe?$AA?$CI?$AA?$CJ?$AA?3?$AA?5?$AAF?$AAa?$AAi?$AAl?$AAe?$AAd?$AA?$CB@ 10001f50     can_common_topaz_v1:canclass.obj
 0001:00000fb0       ??_C@_1DA@IBGPFIHO@?$AAC?$AAA?$AAN?$AAC?$AAl?$AAa?$AAs?$AAs?$AA?3?$AA?3?$AA?$HO?$AAC?$AAA?$AAN?$AAC?$AAl?$AAa?$AAs?$AAs?$AA?5?$AA?9?$AA?$AN?$AA?6?$AA?$AA@ 10001fb0     can_common_topaz_v1:canclass.obj
 0001:00000fe0       ??_C@_1JA@KEPLBFAM@?$AAC?$AAA?$AAN?$AAC?$AAl?$AAa?$AAs?$AAs?$AA?3?$AA?3?$AA?$HO?$AAC?$AAA?$AAN?$AAC?$AAl?$AAa?$AAs?$AAs?$AA?3?$AA?5?$AAR?$AAe?$AAl?$AAe?$AAa?$AAs?$AAe?$AA?5?$AAC?$AAA?$AAN@ 10001fe0     can_common_topaz_v1:canclass.obj
 0001:00001070       ??_C@_1HE@BMLLJCLB@?$AAC?$AAA?$AAN?$AAC?$AAl?$AAa?$AAs?$AAs?$AA?3?$AA?3?$AA?$HO?$AAC?$AAA?$AAN?$AAC?$AAl?$AAa?$AAs?$AAs?$AA?3?$AA?5?$AAR?$AAe?$AAl?$AAe?$AAa?$AAs?$AAe?$AA?5?$AAI?$AAn?$AAt@ 10002070     can_common_topaz_v1:canclass.obj
 0001:000010e8       ??_C@_1LC@OEIFJGMB@?$AAC?$AAA?$AAN?$AAC?$AAl?$AAa?$AAs?$AAs?$AA?3?$AA?3?$AA?$HO?$AAC?$AAA?$AAN?$AAC?$AAl?$AAa?$AAs?$AAs?$AA?3?$AAD?$AAe?$AAl?$AAe?$AAt?$AAe?$AAC?$AAr?$AAi?$AAt?$AAi?$AAc@ 100020e8     can_common_topaz_v1:canclass.obj
 0001:000011a0       ??_C@_1EM@HCNAFH@?$AAE?$AAR?$AAR?$AAO?$AAR?$AA?3?$AA?5?$AAF?$AAa?$AAi?$AAl?$AAe?$AAd?$AA?5?$AAt?$AAo?$AA?5?$AAr?$AAe?$AAl?$AAe?$AAa?$AAs?$AAe?$AA?5?$AAd?$AAw?$AAS?$AAy?$AAs?$AAI?$AAn@ 100021a0     can_common_topaz_v1:canclass.obj
 0001:000011f0       ??_C@_1GK@LIEJBJOP@?$AAC?$AAA?$AAN?$AAC?$AAl?$AAa?$AAs?$AAs?$AA?3?$AA?3?$AA?$HO?$AAC?$AAA?$AAN?$AAC?$AAl?$AAa?$AAs?$AAs?$AA?$CI?$AA?$CJ?$AA?3?$AA?5?$AAR?$AAe?$AAl?$AAe?$AAa?$AAs?$AAi?$AAn?$AAg@ 100021f0     can_common_topaz_v1:canclass.obj
 0001:00001260       ??_C@_1GC@MKFEDHIN@?$AAC?$AAA?$AAN?$AAC?$AAl?$AAa?$AAs?$AAs?$AA?3?$AA?3?$AA?$HO?$AAC?$AAA?$AAN?$AAC?$AAl?$AAa?$AAs?$AAs?$AA?3?$AA?5?$AAR?$AAe?$AAl?$AAe?$AAa?$AAs?$AAe?$AA?5?$AAS?$AAy?$AAs@ 10002260     can_common_topaz_v1:canclass.obj
 0001:000012c4       ??_C@_1DA@EHAAFBPJ@?$AAC?$AAA?$AAN?$AAC?$AAl?$AAa?$AAs?$AAs?$AA?3?$AA?3?$AA?$HO?$AAC?$AAA?$AAN?$AAC?$AAl?$AAa?$AAs?$AAs?$AA?5?$AA?$CL?$AA?$AN?$AA?6?$AA?$AA@ 100022c4     can_common_topaz_v1:canclass.obj
 0001:000012f4       ??_C@_1BK@ODFIPLC@?$AAC?$AAA?$AAN?$AAR?$AAe?$AAs?$AAe?$AAt?$AA?9?$AA?9?$AA?$AN?$AA?6?$AA?$AA@ 100022f4     can_common_topaz_v1:canclass.obj
 0001:00001310       ??_C@_1BK@MFEEPGHC@?$AAC?$AAA?$AAN?$AAR?$AAe?$AAs?$AAe?$AAt?$AA?$CL?$AA?$CL?$AA?$AN?$AA?6?$AA?$AA@ 10002310     can_common_topaz_v1:canclass.obj
 0001:0000132c       ??_C@_1CG@FKGBIGEP@?$AAC?$AAA?$AAN?$AAP?$AAo?$AAw?$AAe?$AAr?$AAH?$AAa?$AAn?$AAd?$AAl?$AAe?$AAr?$AA?9?$AA?$AN?$AA?6?$AA?$AA@ 1000232c     can_common_topaz_v1:canclass.obj
 0001:00001354       ??_C@_1CM@IDLOFHBA@?$AAC?$AAA?$AAN?$AAP?$AAo?$AAw?$AAe?$AAr?$AAH?$AAa?$AAn?$AAd?$AAl?$AAe?$AAr?$AA?$CL?$AA?3?$AA?$CF?$AAd?$AA?$AN?$AA?6?$AA?$AA@ 10002354     can_common_topaz_v1:canclass.obj
 0001:00001380       ??_C@_1EG@JBACIDOL@?$AAC?$AAA?$AAN?$AAS?$AAe?$AAt?$AAM?$AAo?$AAd?$AAe?$AA?5?$AAi?$AAn?$AAd?$AAe?$AAx?$AA?3?$AA?$CF?$AAd?$AA?5?$AAC?$AAA?$AAN?$AA_?$AAM?$AAO?$AAD?$AAE?$AA?3?$AA?$CF?$AAd?$AA?5@ 10002380     can_common_topaz_v1:canclass.obj
 0001:000013c8       ??_C@_1DO@OLAGJECD@?$AA?5?$AAW?$AAr?$AAi?$AAt?$AAe?$AAP?$AAa?$AAc?$AAk?$AAe?$AAt?$AA?5?$AA?5?$AAp?$AAC?$AAA?$AAN?$AAP?$AAk?$AAt?$AA?9?$AA?$DO?$AAI?$AAD?$AA?3?$AA?$CF?$AAx?$AA?$AN?$AA?6?$AA?$AA@ 100023c8     can_common_topaz_v1:canclass.obj
 0001:00001408       ??_C@_1BM@KHBGMODP@?$AAW?$AAr?$AAi?$AAt?$AAe?$AAP?$AAa?$AAc?$AAk?$AAe?$AAt?$AA?$AN?$AA?6?$AA?$AA@ 10002408     can_common_topaz_v1:canclass.obj
 0001:00001428       ??_C@_1HC@BMINOAGE@?$AAR?$AAe?$AAa?$AAd?$AAP?$AAa?$AAc?$AAk?$AAe?$AAt?$AA?5?$AAI?$AAn?$AAd?$AAe?$AAx?$AA?5?$AA?3?$AA?$CF?$AAd?$AA?5?$AAg?$AAi?$AAn?$AAd?$AAe?$AAx?$AA?3?$AA?$CF?$AAd?$AA?5?$AA?5@ 10002428     can_common_topaz_v1:canclass.obj
 0001:0000149c       ??_C@_1DC@FABDFIOO@?$AAC?$AAA?$AAN?$AA_?$AAR?$AAe?$AAa?$AAd?$AA?5?$AAI?$AAM?$AAA?$AAS?$AAK?$AA2?$AA?3?$AA0?$AAx?$AA?3?$AA?$CF?$AAx?$AA?5?$AA?$AN?$AA?6?$AA?$AA@ 1000249c     can_common_topaz_v1:canclass.obj
 0001:000014d0       ??_C@_1DC@GJGLPFKO@?$AAC?$AAA?$AAN?$AA_?$AAR?$AAe?$AAa?$AAd?$AA?5?$AAI?$AAM?$AAA?$AAS?$AAK?$AA1?$AA?3?$AA0?$AAx?$AA?3?$AA?$CF?$AAx?$AA?5?$AA?$AN?$AA?6?$AA?$AA@ 100024d0     can_common_topaz_v1:canclass.obj
 0001:00001504       ??_C@_1CK@EJFNKPCD@?$AAC?$AAA?$AAN?$AA_?$AAR?$AAe?$AAa?$AAd?$AA?5?$AAI?$AAD?$AA?3?$AA0?$AAx?$AA?3?$AA?$CF?$AAx?$AA?5?$AA?$AN?$AA?6?$AA?$AA@ 10002504     can_common_topaz_v1:canclass.obj
 0001:00001530       ??_C@_1BK@EJGEPGLA@?$AAR?$AAe?$AAa?$AAd?$AAP?$AAa?$AAc?$AAk?$AAe?$AAt?$AA?$AN?$AA?6?$AA?$AA@ 10002530     can_common_topaz_v1:canclass.obj
 0001:0000154c       ??_C@_1DG@CAIPPAG@?$AAC?$AAA?$AAN?$AA?3?$AA?3?$AAP?$AAr?$AAo?$AAc?$AAe?$AAs?$AAs?$AAP?$AAa?$AAc?$AAk?$AAe?$AAt?$AAs?$AA?5?$AAF?$AAa?$AAi?$AAl?$AA?$AN?$AA?6?$AA?$AA@ 1000254c     can_common_topaz_v1:canclass.obj
 0001:00001588       ??_C@_1IA@POAIDBLI@?$AAC?$AAA?$AAN?$AAC?$AAl?$AAa?$AAs?$AAs?$AA?3?$AA?3?$AAP?$AAr?$AAo?$AAc?$AAe?$AAs?$AAs?$AAP?$AAa?$AAc?$AAk?$AAe?$AAt?$AA?$CI?$AA?$CJ?$AA?3?$AA?5?$AAS?$AAe?$AAt?$AAt?$AAi@ 10002588     can_common_topaz_v1:canclass.obj
 0001:00001608       ??_C@_1GE@KBOICJKF@?$AAC?$AAA?$AAN?$AAC?$AAl?$AAa?$AAs?$AAs?$AA?3?$AA?3?$AAC?$AAA?$AAN?$AAI?$AAn?$AAt?$AAe?$AAr?$AAr?$AAu?$AAp?$AAt?$AAH?$AAa?$AAn?$AAd?$AAl?$AAe?$AAr?$AA?3?$AA?5?$AAC@ 10002608     can_common_topaz_v1:canclass.obj
 0001:00001670       ??_C@_1GE@LOCFLEIF@?$AAC?$AAA?$AAN?$AAC?$AAl?$AAa?$AAs?$AAs?$AA?3?$AA?3?$AAC?$AAA?$AAN?$AAI?$AAn?$AAt?$AAe?$AAr?$AAr?$AAu?$AAp?$AAt?$AAH?$AAa?$AAn?$AAd?$AAl?$AAe?$AAr?$AA?3?$AA?5?$AAC@ 10002670     can_common_topaz_v1:canclass.obj
 0001:000016d8       ??_C@_1GE@BJDBCLKA@?$AAC?$AAA?$AAN?$AAC?$AAl?$AAa?$AAs?$AAs?$AA?3?$AA?3?$AAC?$AAA?$AAN?$AAI?$AAn?$AAt?$AAe?$AAr?$AAr?$AAu?$AAp?$AAt?$AAH?$AAa?$AAn?$AAd?$AAl?$AAe?$AAr?$AA?3?$AA?5?$AAC@ 100026d8     can_common_topaz_v1:canclass.obj
 0001:00001740       ??_C@_1GC@DFOJGJEK@?$AAC?$AAA?$AAN?$AAC?$AAl?$AAa?$AAs?$AAs?$AA?3?$AA?3?$AAC?$AAA?$AAN?$AAI?$AAn?$AAt?$AAe?$AAr?$AAr?$AAu?$AAp?$AAt?$AAH?$AAa?$AAn?$AAd?$AAl?$AAe?$AAr?$AA?3?$AA?5?$AAC@ 10002740     can_common_topaz_v1:canclass.obj
 0001:000017a8       ??_C@_1GM@GGGBGAGE@?$AAC?$AAA?$AAN?$AAC?$AAl?$AAa?$AAs?$AAs?$AA?3?$AA?3?$AAC?$AAA?$AAN?$AAI?$AAn?$AAt?$AAe?$AAr?$AAr?$AAu?$AAp?$AAt?$AAH?$AAa?$AAn?$AAd?$AAl?$AAe?$AAr?$AA?3?$AAC?$AAA@ 100027a8     can_common_topaz_v1:canclass.obj
 0001:00001818       ??_C@_1GM@HMGCGHIH@?$AAC?$AAA?$AAN?$AAC?$AAl?$AAa?$AAs?$AAs?$AA?3?$AA?3?$AAC?$AAA?$AAN?$AAI?$AAn?$AAt?$AAe?$AAr?$AAr?$AAu?$AAp?$AAt?$AAH?$AAa?$AAn?$AAd?$AAl?$AAe?$AAr?$AA?3?$AA?5?$AAC@ 10002818     can_common_topaz_v1:canclass.obj
 0001:00001888       ??_C@_1HK@KFLFIGBI@?$AAC?$AAA?$AAN?$AAC?$AAl?$AAa?$AAs?$AAs?$AA?3?$AA?3?$AAC?$AAA?$AAN?$AAI?$AAn?$AAt?$AAe?$AAr?$AAr?$AAu?$AAp?$AAt?$AAH?$AAa?$AAn?$AAd?$AAl?$AAe?$AAr?$AA?3?$AA?5?$AAC@ 10002888     can_common_topaz_v1:canclass.obj
 0001:00001908       ??_C@_1HO@PHLHHDCP@?$AAC?$AAA?$AAN?$AAC?$AAl?$AAa?$AAs?$AAs?$AA?3?$AA?3?$AAC?$AAA?$AAN?$AAI?$AAn?$AAt?$AAe?$AAr?$AAr?$AAu?$AAp?$AAt?$AAH?$AAa?$AAn?$AAd?$AAl?$AAe?$AAr?$AA?3?$AA?5?$AA?$EA@ 10002908     can_common_topaz_v1:canclass.obj
 0001:00001988       ??_C@_1HK@IINIJDPG@?$AAC?$AAA?$AAN?$AAC?$AAl?$AAa?$AAs?$AAs?$AA?3?$AA?3?$AAC?$AAA?$AAN?$AAI?$AAn?$AAt?$AAe?$AAr?$AAr?$AAu?$AAp?$AAt?$AAH?$AAa?$AAn?$AAd?$AAl?$AAe?$AAr?$AA?3?$AA?5?$AAC@ 10002988     can_common_topaz_v1:canclass.obj
 0001:00001a08       ??_C@_1HI@CPPKDMLB@?$AAC?$AAA?$AAN?$AAC?$AAl?$AAa?$AAs?$AAs?$AA?3?$AA?3?$AAC?$AAA?$AAN?$AAI?$AAn?$AAt?$AAe?$AAr?$AAr?$AAu?$AAp?$AAt?$AAH?$AAa?$AAn?$AAd?$AAl?$AAe?$AAr?$AA?3?$AA?5?$AAC@ 10002a08     can_common_topaz_v1:canclass.obj
 0001:00001a80       ??_C@_1EC@CBNOJBDP@?$AAC?$AAA?$AAN?$AAI?$AAn?$AAt?$AAe?$AAr?$AAr?$AAu?$AAp?$AAt?$AAH?$AAa?$AAn?$AAd?$AAl?$AAe?$AAr?$AA?5?$AAE?$AAC?$AAR?$AA?3?$AA0?$AAx?$AA?3?$AA?$CF?$AAx?$AA?5?$AA?$AN?$AA?6@ 10002a80     can_common_topaz_v1:canclass.obj
 0001:00001ac8       ??_C@_1EC@FOLFOOAC@?$AAC?$AAA?$AAN?$AAI?$AAn?$AAt?$AAe?$AAr?$AAr?$AAu?$AAp?$AAt?$AAH?$AAa?$AAn?$AAd?$AAl?$AAe?$AAr?$AA?5?$AAE?$AAS?$AAR?$AA?3?$AA0?$AAx?$AA?3?$AA?$CF?$AAx?$AA?5?$AA?$AN?$AA?6@ 10002ac8     can_common_topaz_v1:canclass.obj
 0001:00001b0c       ??_C@_1DA@ECIBNJLH@?$AAC?$AAA?$AAN?$AA_?$AAI?$AAn?$AAt?$AAr?$AAT?$AAh?$AAr?$AAe?$AAa?$AAd?$AA?5?$AAE?$AAn?$AAt?$AAe?$AAr?$AA?5?$AA?$AN?$AA?6?$AA?$AA@ 10002b0c     can_common_topaz_v1:canclass.obj
 0001:00001b5c       CANConfigureGPIO           10002b5c f   bspcan.obj
 0001:00001e34       BSPCANClockConfig          10002e34 f   bspcan.obj
 0001:00001f28       BSPCANConfigureGPIO        10002f28 f   bspcan.obj
 0001:00001f78       BSPGetCANBaseRegAddr       10002f78 f   bspcan.obj
 0001:00001fe0       BSPGetCANIRQ               10002fe0 f   bspcan.obj
 0001:00002040       BSPSetCanPowerEnable       10003040 f   bspcan.obj
 0001:000020f4       ?CAN_Init@@YAKPBG@Z        100030f4 f   can_common_topaz_v1:can_io.obj
 0001:000022ec       ?CAN_Deinit@@YAHK@Z        100032ec f   can_common_topaz_v1:can_io.obj
 0001:000023ec       ?CAN_Open@@YAKKKK@Z        100033ec f   can_common_topaz_v1:can_io.obj
 0001:00002498       ?CAN_Close@@YAHK@Z         10003498 f   can_common_topaz_v1:can_io.obj
 0001:00002540       ?CAN_PowerDown@@YAXK@Z     10003540 f   can_common_topaz_v1:can_io.obj
 0001:00002550       ?CAN_PowerUp@@YAXXZ        10003550 f   can_common_topaz_v1:can_io.obj
 0001:00002554       ?CAN_Read@@YAKKPAXK@Z      10003554 f   can_common_topaz_v1:can_io.obj
 0001:00002578       ?CAN_Write@@YAKKPBXK@Z     10003578 f   can_common_topaz_v1:can_io.obj
 0001:0000259c       ?CAN_Seek@@YAKKJG@Z        1000359c f   can_common_topaz_v1:can_io.obj
 0001:000025c8       ?CAN_IOControl@@YAHKKPAEK0KPAK@Z 100035c8 f   can_common_topaz_v1:can_io.obj
 0001:00003618       ?CAN_DllEntry@@YAHPAXK0@Z  10004618 f   can_common_topaz_v1:can_io.obj
 0001:000036e4       ??_GCANClass@@QAAPAXI@Z    100046e4 f i can_common_topaz_v1:can_io.obj
 0001:00003724       ??1MarshalledBuffer_t@@QAA@XZ 10004724 f i can_common_topaz_v1:can_io.obj
 0001:0000373c       ??0MarshalledBuffer_t@@QAA@PAXKKHH@Z 1000473c f i can_common_topaz_v1:can_io.obj
 0001:0000378c       ?Reset@MarshalledBuffer_t@@AAAXXZ 1000478c f i can_common_topaz_v1:can_io.obj
 0001:000037c8       ?Marshal@MarshalledBuffer_t@@QAAJPAXKKHH@Z 100047c8 f i can_common_topaz_v1:can_io.obj
 0001:000038c8       ?Unmarshal@MarshalledBuffer_t@@QAAJXZ 100048c8 f i can_common_topaz_v1:can_io.obj
 0001:00003994       ?ptr@MarshalledBuffer_t@@QBAPAXXZ 10004994 f i can_common_topaz_v1:can_io.obj
 0001:000039e0       ??_GMarshalledBuffer_t@@QAAPAXI@Z 100049e0 f i can_common_topaz_v1:can_io.obj
 0001:00003a20       ??0?$Buffer_t@VDuplicateTraits_t@detail@marshal@ce@@@detail@marshal@ce@@QAA@PAXKK@Z 10004a20 f i can_common_topaz_v1:can_io.obj
 0001:00003a70       ?ptr@?$Buffer_t@VDuplicateTraits_t@detail@marshal@ce@@@detail@marshal@ce@@QBAPAXXZ 10004a70 f i can_common_topaz_v1:can_io.obj
 0001:00003a9c       ??1?$Buffer_t@VDuplicateTraits_t@detail@marshal@ce@@@detail@marshal@ce@@UAA@XZ 10004a9c f i can_common_topaz_v1:can_io.obj
 0001:00003ac4       ??_G?$Buffer_t@VDuplicateTraits_t@detail@marshal@ce@@@detail@marshal@ce@@UAAPAXI@Z 10004ac4 f i can_common_topaz_v1:can_io.obj
 0001:00003ac4       ??_E?$Buffer_t@VDuplicateTraits_t@detail@marshal@ce@@@detail@marshal@ce@@UAAPAXI@Z 10004ac4 f i can_common_topaz_v1:can_io.obj
 0001:00003b04       ?Reset@?$Buffer_t@VDuplicateTraits_t@detail@marshal@ce@@@detail@marshal@ce@@AAAXXZ 10004b04 f i can_common_topaz_v1:can_io.obj
 0001:00003b44       ?Free@?$Buffer_t@VDuplicateTraits_t@detail@marshal@ce@@@detail@marshal@ce@@QAAJXZ 10004b44 f i can_common_topaz_v1:can_io.obj
 0001:00003bdc       ?free@DuplicateTraits_t@detail@marshal@ce@@QBAJPAX0KK@Z 10004bdc f i can_common_topaz_v1:can_io.obj
 0001:00003c18       ?Allocate@?$Buffer_t@VDuplicateTraits_t@detail@marshal@ce@@@detail@marshal@ce@@QAAJPAXKK@Z 10004c18 f i can_common_topaz_v1:can_io.obj
 0001:00003cc8       ?alloc@DuplicateTraits_t@detail@marshal@ce@@QBAJPAPAXPAXKK@Z 10004cc8 f i can_common_topaz_v1:can_io.obj
 0001:00003d04       ?GetIndex@@YAHI@Z          10004d04 f   can_common_topaz_v1:canclass.obj
 0001:00003d70       ??0CANClass@@QAA@I@Z       10004d70 f   can_common_topaz_v1:canclass.obj
 0001:000045a8       ??1CANClass@@QAA@XZ        100055a8 f   can_common_topaz_v1:canclass.obj
 0001:000048d4       ?CANEnableTLPRIOMode@CANClass@@QAAHH@Z 100058d4 f   can_common_topaz_v1:canclass.obj
 0001:0000492c       ?CANReset@CANClass@@QAAHXZ 1000592c f   can_common_topaz_v1:canclass.obj
 0001:000049e0       ?CANPowerHandler@CANClass@@QAAHH@Z 100059e0 f   can_common_topaz_v1:canclass.obj
 0001:00004b04       ?CANSetMode@CANClass@@QAAXKW4_CAN_MODE@@@Z 10005b04 f   can_common_topaz_v1:canclass.obj
 0001:00004c04       ?WritePacket@CANClass@@QAAHPAUCAN_PACKET@@H@Z 10005c04 f   can_common_topaz_v1:canclass.obj
 0001:00004f88       ?ReadPacket@CANClass@@QAAHPAUCAN_PACKET@@H@Z 10005f88 f   can_common_topaz_v1:canclass.obj
 0001:000053c0       ?ProcessPackets@CANClass@@QAAHQAUCAN_PACKET@@H@Z 100063c0 f   can_common_topaz_v1:canclass.obj
 0001:0000556c       ?CANIST@CANClass@@CAXPAX@Z 1000656c f   can_common_topaz_v1:canclass.obj
 0001:00005598       ?CANInterruptHandler@CANClass@@AAAXI@Z 10006598 f   can_common_topaz_v1:canclass.obj
 0001:00005d10       PulseEvent                 10006d10 f i can_common_topaz_v1:canclass.obj
 0001:00005d44       GetCurrentThread           10006d44 f i can_common_topaz_v1:canclass.obj
 0001:00005d5c       SetEvent                   10006d5c f i can_common_topaz_v1:canclass.obj
 0001:00005d90       NKDbgPrintfW               10006d90 f   coredll:COREDLL.dll
 0001:00005da0       RegCloseKey                10006da0 f   coredll:COREDLL.dll
 0001:00005db0       RegQueryValueExW           10006db0 f   coredll:COREDLL.dll
 0001:00005dc0       OpenDeviceKey              10006dc0 f   coredll:COREDLL.dll
 0001:00005dd0       GetLastError               10006dd0 f   coredll:COREDLL.dll
 0001:00005de0       CeAllocAsynchronousBuffer  10006de0 f   coredll:COREDLL.dll
 0001:00005df0       CeOpenCallerBuffer         10006df0 f   coredll:COREDLL.dll
 0001:00005e00       CeCloseCallerBuffer        10006e00 f   coredll:COREDLL.dll
 0001:00005e10       CeFreeAsynchronousBuffer   10006e10 f   coredll:COREDLL.dll
 0001:00005e20       DisableThreadLibraryCalls  10006e20 f   coredll:COREDLL.dll
 0001:00005e30       RegisterDbgZones           10006e30 f   coredll:COREDLL.dll
 0001:00005e40       CeFreeDuplicateBuffer      10006e40 f   coredll:COREDLL.dll
 0001:00005e50       CeAllocDuplicateBuffer     10006e50 f   coredll:COREDLL.dll
 0001:00005e60       InitializeCriticalSection  10006e60 f   coredll:COREDLL.dll
 0001:00005e70       CeSetThreadPriority        10006e70 f   coredll:COREDLL.dll
 0001:00005e80       CreateThread               10006e80 f   coredll:COREDLL.dll
 0001:00005e90       InterruptInitialize        10006e90 f   coredll:COREDLL.dll
 0001:00005ea0       KernelIoControl            10006ea0 f   coredll:COREDLL.dll
 0001:00005eb0       CreateEventW               10006eb0 f   coredll:COREDLL.dll
 0001:00005ec0       CloseHandle                10006ec0 f   coredll:COREDLL.dll
 0001:00005ed0       InterruptDisable           10006ed0 f   coredll:COREDLL.dll
 0001:00005ee0       EventModify                10006ee0 f   coredll:COREDLL.dll
 0001:00005ef0       InterruptDone              10006ef0 f   coredll:COREDLL.dll
 0001:00005f00       WaitForSingleObject        10006f00 f   coredll:COREDLL.dll
 0001:00005f10       LeaveCriticalSection       10006f10 f   coredll:COREDLL.dll
 0001:00005f20       EnterCriticalSection       10006f20 f   coredll:COREDLL.dll
 0001:00005f30       MmMapIoSpace               10006f30 f   ceddk:CEDDK.dll
 0001:00005f40       MmUnmapIoSpace             10006f40 f   ceddk:CEDDK.dll
 0001:00005f50       DDKIomuxSelectInput        10006f50 f   cspddk:CSPDDK.dll
 0001:00005f60       DDKGpioWriteDataPin        10006f60 f   cspddk:CSPDDK.dll
 0001:00005f70       DDKGpioSetConfig           10006f70 f   cspddk:CSPDDK.dll
 0001:00005f80       DDKIomuxSetPadConfig       10006f80 f   cspddk:CSPDDK.dll
 0001:00005f90       DDKIomuxSetPinMux          10006f90 f   cspddk:CSPDDK.dll
 0001:00005fa0       DDKClockSetGatingMode      10006fa0 f   cspddk:CSPDDK.dll
 0001:00005fb0       DllMain                    10006fb0 f   corelib0:dllmain.obj
 0001:00005fe8       _DllMainCRTStartup         10006fe8 f   corelib0:pegdmain.obj
 0001:00006180       __security_init_cookie     10007180 f   corelib0:seccinit.obj
 0001:00006218       exit                       10007218 f   corelib0:cexit.obj
 0001:0000633c       _exit                      1000733c f   corelib0:cexit.obj
 0001:0000635c       _cexit                     1000735c f   corelib0:cexit.obj
 0001:00006374       _c_exit                    10007374 f   corelib0:cexit.obj
 0001:0000638c       _initterm                  1000738c f   corelib0:crt0dat.obj
 0001:000063d8       _cinit                     100073d8 f   corelib0:crt0dat.obj
 0001:00006408       __crt_ExitProcess          10007408 f   corelib0:exitproc_proxy.obj
 0001:00006434       GetCurrentProcess          10007434 f i corelib0:exitproc_proxy.obj
 0001:0000644c       _onexit                    1000744c f   corelib0:onexit.obj
 0001:00006628       atexit                     10007628 f   corelib0:onexit.obj
 0001:00006678       ??2@YAPAXI@Z               10007678 f   corelib1:COREDLL.dll
 0001:00006688       ??3@YAXPAX@Z               10007688 f   corelib1:COREDLL.dll
 0001:00006698       memset                     10007698 f   corelib1:COREDLL.dll
 0001:000066a8       __C_specific_handler       100076a8 f   corelib1:COREDLL.dll
 0001:000066b8       _XcptFilter                100076b8 f   corelib1:COREDLL.dll
 0001:000066c8       __security_gen_cookie2     100076c8 f   corelib1:COREDLL.dll
 0001:000066d8       free                       100076d8 f   corelib1:COREDLL.dll
 0001:000066e8       realloc                    100076e8 f   corelib1:COREDLL.dll
 0001:000066f8       malloc                     100076f8 f   corelib1:COREDLL.dll
 0001:00006708       _msize                     10007708 f   corelib1:COREDLL.dll
 0001:00006718       TerminateProcess           10007718 f   coredll:COREDLL.dll
 0001:00006770       __IMPORT_DESCRIPTOR_COREDLL 10007770     coredll:COREDLL.dll
 0001:00006784       __IMPORT_DESCRIPTOR_CEDDK  10007784     ceddk:CEDDK.dll
 0001:00006798       __IMPORT_DESCRIPTOR_CSPDDK 10007798     cspddk:CSPDDK.dll
 0001:000067ac       __NULL_IMPORT_DESCRIPTOR   100077ac     coredll:COREDLL.dll
 0002:00000000       __imp_MmMapIoSpace         10008000     ceddk:CEDDK.dll
 0002:00000004       __imp_MmUnmapIoSpace       10008004     ceddk:CEDDK.dll
 0002:00000008       \177CEDDK_NULL_THUNK_DATA  10008008     ceddk:CEDDK.dll
 0002:0000000c       __imp_OpenDeviceKey        1000800c     coredll:COREDLL.dll
 0002:00000010       __imp_GetLastError         10008010     coredll:COREDLL.dll
 0002:00000014       __imp_CeAllocAsynchronousBuffer 10008014     coredll:COREDLL.dll
 0002:00000018       __imp_CeOpenCallerBuffer   10008018     coredll:COREDLL.dll
 0002:0000001c       __imp_CeCloseCallerBuffer  1000801c     coredll:COREDLL.dll
 0002:00000020       __imp_CeFreeAsynchronousBuffer 10008020     coredll:COREDLL.dll
 0002:00000024       __imp_DisableThreadLibraryCalls 10008024     coredll:COREDLL.dll
 0002:00000028       __imp_RegisterDbgZones     10008028     coredll:COREDLL.dll
 0002:0000002c       __imp_CeFreeDuplicateBuffer 1000802c     coredll:COREDLL.dll
 0002:00000030       __imp_CeAllocDuplicateBuffer 10008030     coredll:COREDLL.dll
 0002:00000034       __imp_InitializeCriticalSection 10008034     coredll:COREDLL.dll
 0002:00000038       __imp_RegQueryValueExW     10008038     coredll:COREDLL.dll
 0002:0000003c       __imp_CreateThread         1000803c     coredll:COREDLL.dll
 0002:00000040       __imp_InterruptInitialize  10008040     coredll:COREDLL.dll
 0002:00000044       __imp_KernelIoControl      10008044     coredll:COREDLL.dll
 0002:00000048       __imp_CreateEventW         10008048     coredll:COREDLL.dll
 0002:0000004c       __imp_CloseHandle          1000804c     coredll:COREDLL.dll
 0002:00000050       __imp_InterruptDisable     10008050     coredll:COREDLL.dll
 0002:00000054       __imp_EventModify          10008054     coredll:COREDLL.dll
 0002:00000058       __imp_InterruptDone        10008058     coredll:COREDLL.dll
 0002:0000005c       __imp_WaitForSingleObject  1000805c     coredll:COREDLL.dll
 0002:00000060       __imp_LeaveCriticalSection 10008060     coredll:COREDLL.dll
 0002:00000064       __imp_EnterCriticalSection 10008064     coredll:COREDLL.dll
 0002:00000068       __imp_RegCloseKey          10008068     coredll:COREDLL.dll
 0002:0000006c       __imp_CeSetThreadPriority  1000806c     coredll:COREDLL.dll
 0002:00000070       __imp_NKDbgPrintfW         10008070     coredll:COREDLL.dll
 0002:00000074       __imp__msize               10008074     corelib1:COREDLL.dll
 0002:00000078       __imp_malloc               10008078     corelib1:COREDLL.dll
 0002:0000007c       __imp_realloc              1000807c     corelib1:COREDLL.dll
 0002:00000080       __imp_free                 10008080     corelib1:COREDLL.dll
 0002:00000084       __imp___security_gen_cookie2 10008084     corelib1:COREDLL.dll
 0002:00000088       __imp__XcptFilter          10008088     corelib1:COREDLL.dll
 0002:0000008c       __imp___C_specific_handler 1000808c     corelib1:COREDLL.dll
 0002:00000090       __imp_??2@YAPAXI@Z         10008090     corelib1:COREDLL.dll
 0002:00000094       __imp_??3@YAXPAX@Z         10008094     corelib1:COREDLL.dll
 0002:00000098       __imp_memset               10008098     corelib1:COREDLL.dll
 0002:0000009c       __imp_TerminateProcess     1000809c     coredll:COREDLL.dll
 0002:000000a0       \177COREDLL_NULL_THUNK_DATA 100080a0     coredll:COREDLL.dll
 0002:000000a4       __imp_DDKIomuxSetPinMux    100080a4     cspddk:CSPDDK.dll
 0002:000000a8       __imp_DDKIomuxSetPadConfig 100080a8     cspddk:CSPDDK.dll
 0002:000000ac       __imp_DDKGpioSetConfig     100080ac     cspddk:CSPDDK.dll
 0002:000000b0       __imp_DDKGpioWriteDataPin  100080b0     cspddk:CSPDDK.dll
 0002:000000b4       __imp_DDKIomuxSelectInput  100080b4     cspddk:CSPDDK.dll
 0002:000000b8       __imp_DDKClockSetGatingMode 100080b8     cspddk:CSPDDK.dll
 0002:000000bc       \177CSPDDK_NULL_THUNK_DATA 100080bc     cspddk:CSPDDK.dll
 0002:000000c0       dpCurSettings              100080c0     can_common_topaz_v1:can_io.obj
 0002:00000504       __security_cookie          10008504     corelib0:seccinit.obj
 0002:00000508       __security_cookie_complement 10008508     corelib0:seccinit.obj
 0002:0000050c       _exitflag                  1000850c     corelib0:cexit.obj
 0002:00000510       __onexitend                10008510     <common>
 0002:00000514       __onexitbegin              10008514     <common>
 0002:00000518       _pRawDllMain               10008518     <common>

 entry point at        0001:00005fe8

 Static symbols

 0001:00006038       _DllMainCRTStartupHelper   10007038 f   corelib0:pegdmain.obj
 0001:00006238       doexit                     10007238 f   corelib0:cexit.obj
